:100000001F3062000A3044298C00030E83018D00EA
:1000100004088F000A088E008A01512982070C34D7
:100020000C340A3400340B340C34073408340934EB
:100030000C340434053406340C34013402340334F3
:1000400003343A0892003430930012089302031CE0
:1000500068280A0896008A0112083220C200160891
:100060008A0068288207FC347C343C341C340C340D
:1000700004348434C434E434F4344034503420340C
:100080001034C034A83490346034783418342834B0
:1000900070348834D0340834A034F0346834D83420
:1000A000B03430344834E0349834B834C8349434FC
:1000B0008C3432345634CE344A3416345434863484
:1000C000E234B434B634143444345834E834383474
:1000D000542A480892000630930012089302031C29
:1000E00082280A0896008A0112087A20C50016089C
:1000F0008A008228820729340A341A34243432349C
:1001000035341134C92A4808920006309300120889
:100110009302031C9C280A0896008A011208942066
:10012000C60016088A009C288207003400340A346E
:100130000034003400342434CA2A9B131208900778
:1001400001300318910703189B1713089107031830
:10015000ED280034E320970C960C03189D20910C99
:10016000900C950C940C9A03031DAB281008920078
:100170001104031D9B171108930014089000150823
:1001800091000034E320940195010310960D970D22
:10019000940D950D13081502031DD02812081402A2
:1001A000031CD92812089402031C95031308950216
:1001B0000314900D910D9A03031DC5281408920095
:1001C00015089300003410309A009B131008960015
:1001D000110897009001910100348030EF289B04B2
:1001E000003483168818F2280812831208000B08BE
:1001F00090008B139A008316081555308900AA3099
:1002000089008814081183120800831608148312C9
:10021000080083160608831298000F3066007030BD
:1002200096000430970016088600000000000609BA
:100230000F39031D27290314960C9703031D132957
:10024000900110080E20800018086600003491000C
:1002500090010430961F2F299007960D2A29900AA5
:1002600011182129910C2F2903109007101C3B29EC
:10027000553090063D29AA309106900D910D3D080C
:100280009007333A910700346500F1306600313051
:100290001E3E84008001E13E031D482929162417D3
:1002A000C82AA00B55292108A00009302002031DEF
:1002B0005A290510AF0AAF0B7C29B31E7C29331ACB
:1002C0006829061868293716A501A401A4148F29E6
:1002D000851971292F153316B717B31D7229B3115C
:1002E0007929B311331E7C29061879291C30AF00F7
:1002F000B315A501A401A414A403240A0319A5039A
:1003000024082504031985299B292608A400270809
:10031000A500B5032F198F29051133109129051553
:100320003314AF1897292F1D97292108A000031017
:10033000AD0CAE0CAF0C331CA22920082102031D0A
:10034000A22905140B11B4030F0884000E088A00BB
:100350000D0E83008C0E0C0E09008B1790228B174C
:10036000B030C200FE222908C700B1230108BD0039
:10037000F130860018308B00331E6300A0308B00F4
:10038000B31671222808C700B123B31238089000B1
:10039000900A900303199B2A900303196B2B900377
:1003A0000319712B90030319772B900303197D2BED
:1003B000900303198F2B90030319902B90030319BB
:1003C000942B90030319AE2B90030319AC2B9003CD
:1003D0000319AF2990030319F02990030319B829D1
:1003E0002908C700B123AC30C200FE2290222A089F
:1003F000BB002B08BC003312B901C3010530C40097
:100400003830840009210A303802031D082AAD293A
:10041000B31BEA2B09303802031D0F2AA90A083042
:100420003802031D142AA903D4232908C700B123C5
:100430004908013EB5004408031D1F2A2D223E082D
:100440004302031D242AAD29352235080319292A20
:10045000252A0223C403F723002AC30A05304A07CA
:100460004907B5000530C4000034B90A391BB90189
:10047000F1203908890005210808BD00CA233B087E
:1004800090003C0891004508920000309300C22083
:100490001208900013089100460892000030930063
:1004A0009D201008BA0021284208803A0319682AC2
:1004B000C21F622AB0176C22B0176C22B0176C22D0
:1004C0006C22652AB0176C226C220310C20D542ACC
:1004D000321908006C22682A0310B00CB10CB20C5F
:1004E00008000330B700B31E772A331AB717340851
:1004F00003197B2A772A383084000921B603360A8B
:100500000319B70336083704031D872A8D2A0C30D8
:100510003802031D8C2A772A0034B31A33120800DC
:100520000310470C223CB600B40AB40B942AB4035F
:10053000B60B942A0800E030C200FE227122B803F4
:1005400008303802031CA72A0319A72AAF2906304E
:100550003802031DAC2ADD2A07303802031DB12AF8
:10056000BF2BB819E12B3808133EBA00FD2238081A
:10057000483E9F00712209303802031CC22A031929
:10058000C22AAF291F08840038088000A8239022BF
:10059000692883284C0ABE008301BE0DBE0DCC0A1B
:1005A0004C0EBE07CC0303104D0D203CA1004B0A9E
:1005B000A8000310A80DA80DB329B901C830C200C6
:1005C000FE223830840009210A303802031DE92A4E
:1005D000AF29B80BE12A0108BD00CA233B08AC00D3
:1005E000391BAD29F120390889002C088800F72033
:1005F0008B1715238B13B90AE12A532254220223A5
:10060000F72300343008AD00B0013108AE00B1016D
:100610003208AF00B20108002A08AC00152390226E
:100620002B08AC001423003490222C0890000030DA
:1006300091006430920000309300C2201008BA008C
:10064000FD2290222C08900000309100643092002E
:1006500000309300C22012089000130891000A3065
:10066000920000309300C2201008BA00FD222C082E
:100670009000003091000A30920000309300C220B8
:1006800012089000130891001008BA009022FD2271
:100690000034A023643090000030910038089200AC
:1006A00000309300AA201008AC00A0230A3090006C
:1006B000003091003808920000309300AA202C08E6
:1006C0009200003093009D201008AC00A0232C085D
:1006D0003807AC0000342208AA002308AB000C2322
:1006E000AD293F08AA004008AB000C23AD294E08F5
:1006F000AA004F08AB000C23AD29CA233B08AA006F
:100700003C08AB003F08A2004008A3004E08BF0011
:100710004F08C0002A08CE002B08CF00AF297B2B42
:100720002908AC002223B3291030C200FE22AC01FC
:1007300055232C0803199E2B2C08A900D423B32978
:10074000712209303802031CA82B0319A82BB80109
:100750003808BA00FD220034A90AA90AA903D42343
:10076000AF293E3090004930910047089200003098
:100770009300C2201008A6001108A70000346030C2
:10078000C200FE2249232C08AA0049232C08AB00F2
:100790009022822B3B0890003C08910034211008E5
:1007A000BB001108BC000034043029020318DC2B04
:1007B0000319DC2B0430A900291F08003F30A900D1
:1007C00008003308803AB300B31FAF293030C200AD
:1007D000FE22B3294308AC000310AC0C0310AC0C90
:1007E0002C0829079B1303189B17C700172A0030F2
:1007F0002F02031CFE2B0319FE2BF72B0034FF2BBB
:08400000FF3FFF3FFF3FFF3FC0
:02400E00FA3F77
:10420000FF00FF00FF00FF00FF00FF00FF00FF00B6
:10421000FF00FF00FF00FF00FF00FF00FF00FF00A6
:10422000FF00FF00FF00FF00FF00FF00FF00FF0096
:10423000FF00FF00FF00FF00FF00FF00FF00FF0086
:10424000FF00FF00FF00FF00FF00FF00FF00FF0076
:10425000FF00FF00FF00FF00FF00FF00FF00FF0066
:10426000FF00FF00FF00FF00FF00FF00FF00FF0056
:10427000FF00FF00FF00FF00FF00FF00FF00FF0046
:00000001FF
